:020000040800F2
:10000000C0260020D10100086F0C0008110C000868
:100010006D0C0008FB020008910D000800000000B4
:10002000000000000000000000000000730C000849
:10003000FD02000800000000710C0008750C0008AB
:10004000EB010008EB010008EB010008EB010008E0
:10005000EB010008EB010008EB010008EB010008D0
:10006000EB010008EB010008EB010008EB010008C0
:10007000EB010008EB010008EB010008EB010008B0
:10008000EB010008EB010008EB010008EB010008A0
:10009000EB010008EB010008EB010008EB01000890
:1000A000EB010008EB010008EB010008EB01000880
:1000B000EB010008EB010008EB010008EB01000870
:1000C000EB010008EB010008EB010008EB01000860
:1000D000EB010008EB010008EB010008EB01000850
:1000E000EB010008EB010008EB010008EB01000840
:1000F000EB010008EB010008EB010008EB01000830
:10010000EB010008EB010008EB010008EB0100081F
:10011000EB010008EB010008EB010008EB0100080F
:10012000EB010008EB010008EB010008EB010008FF
:1001300000F002F800F03CF80AA090E8000C8244BD
:100140008344AAF10107DA4501D100F031F8AFF29A
:10015000090EBAE80F0013F0010F18BFFB1A43F0A5
:1001600001031847D00C0000F00C0000103A24BF27
:1001700078C878C1FAD8520724BF30C830C144BF0C
:1001800004680C607047000000230024002500264E
:10019000103A28BF78C1FBD8520728BF30C148BFEA
:1001A0000B6070471FB500F05DF81FBD10B510BDA6
:1001B00000F075F81146FFF7F5FF00F015FE00F0AE
:1001C00093F803B4FFF7F2FF03BC00F061F80000FE
:1001D0000948804709480047FEE7FEE7FEE7FEE7DB
:1001E000FEE7FEE7FEE7FEE7FEE7FEE70448054917
:1001F000054A064B70470000D70C00083101000883
:10020000C0000020C0260020C0120020C012002024
:100210004FF0000200B5134694469646203922BF9F
:10022000A0E80C50A0E80C50B1F12001BFF4F7AFEA
:10023000090728BFA0E80C5048BF0CC05DF804EBCC
:10024000890028BF40F8042B08BF704748BF20F83A
:10025000022B11F0804F18BF00F8012B7047704738
:100260007047704770B5064C7C44064D7D4403E0F2
:10027000206820448047241DAC42F9D170BD0000A5
:10028000E80B0000E80B0000004870476000002009
:1002900001491820ABBEFEE72600020070477546F4
:1002A000FFF7F2FFAE4605006946534620F007000F
:1002B000854618B020B5FFF799FFBDE820404FF004
:1002C00000064FF000074FF000084FF0000B21F040
:1002D0000701AC46ACE8C009ACE8C009ACE8C0090D
:1002E000ACE8C0098D46704710B50446AFF30080F6
:1002F0002046BDE81040FFF764BFFEE7704772B6C6
:10030000FEE700002DE9F84FDFF8C891002409F15D
:10031000040A0AF1040B23460F270BF1040ED1E067
:100320000125A54006EA0502AA4276D1DFF8A8C158
:100330004E68A6EB0C0866452BD00DDC032E34D09E
:1003400005DC36B3012E19D0022E2FD11BE0112E61
:1003500016D0122E2AD119E0B8F5881F19D006DC64
:10036000B8F5803F15D0B8F5801F1FD111E0B8F562
:10037000001F0ED0B8F5041F18D10AE0CB6815E0B5
:10038000CB681B1D12E0CB6808330FE0CB680C3341
:100390000CE08B682BB1012B4FF0080303D04561B3
:1003A00004E0042302E0056100E00023FF2A01D8F5
:1003B000064601E000F104064FEA840501D9A5F1E3
:1003C0002005D6F8008007FA05FC28EA0C0803FA95
:1003D00005F548EA0508C6F800804D68ED0070D5BF
:1003E0003E4DAE6946F00106AE61AD6924F00306EC
:1003F00005F0010500953A4D06EB050CDCF80850B8
:10040000A607360F07FA06F825EA0805DFF8D480B4
:10041000404503D14FF0000825E052E0DFF8C880E6
:10042000404502D14FF001081DE0DFF8C080404593
:1004300002D14FF0020816E0DFF8B480404502D147
:100440004FF003080FE0DFF8AC80404502D14FF0D9
:10045000040808E0DFF8A080404502D14FF005080D
:1004600001E04FF0060808FA06F848EA0508CCF85B
:1004700008804D68D9F80060ED034D4601D516435C
:1004800000E096432E604D68DAF80060AD035546F3
:1004900001D5164300E096432E604D68DBF80060FE
:1004A000ED025D4601D5164300E096432E604D688F
:1004B000DEF80060AD02754601D5164300E09643B4
:1004C0002E60641C0A681646E2407FF429AFBDE83E
:1004D000F88F0000000401400000111000100240DD
:1004E0000000014000080140000C014000100140E4
:1004F0000014014000180140001C014001488068C0
:100500007047000000000020024881680278114412
:100510008160704700000020074810B5016841F075
:1005200010010160032000F067F8002000F006F8D9
:1005300000F024F8002010BD0020024070B50D4DE1
:1005400004464FF47A712878B1FBF0F00A49096843
:10055000B1FBF0F000F0DEFA48B9102C07D200220F
:100560002146501E00F028F800206C6070BD01206C
:1005700070BD0000000000200C0000200C4808B5F1
:10058000816941F001018161816901F001010091FE
:10059000C16941F08051C161C06900F08050009094
:1005A0000448416821F0E06141F00071416008BDFC
:1005B0000010024000000140F0B40E4B1B680C46D6
:1005C000C3F30223C3F10705042D00D90425191D27
:1005D000072901D2002300E0DB1E012606FA05F1FF
:1005E000491E214099409E40761E16403143F0BC82
:1005F00000F0E2BB0CED00E0064900F007020868DD
:100600004FF6FF03184040EA0220034A10430860F7
:10061000704700000CED00E00000FA052DE9F047FE
:100620000F46050061D0434E306800F00700B84225
:1006300009D2306820F0070038433060306800F09D
:100640000700B84251D128683B4C810712D54007BA
:1006500003D5606840F4E06060602878000703D547
:10066000606840F4605060606068A96820F0F00045
:10067000084360602878C00728D06868012810D037
:100680002168022810D0890700292EDA616821F03C
:10069000030101436160FFF731FF804641F2883971
:1006A0000DE021688903EFE78901EDE7FFF726FFF9
:1006B000A0EB0801494502D90320BDE8F087606836
:1006C000696800F00C00B0EB810FEFD1306800F0EA
:1006D0000700B8420BD9306820F00700384330607B
:1006E000306800F00700B84201D00120E5E7287823
:1006F000400705D56068E96820F4E0600843606061
:100700002878000706D56068296920F4605040EA1F
:10071000C100606000F038F86168084AC1F3031155
:10072000515CC8400649086006480068FFF706FFAC
:100730000020C2E70020024000100240020E000824
:100740000C000020040000200448054900684968A6
:10075000044AC1F30221515CC84070470C000020DC
:1007600000100240120E000804480549006849685C
:10077000044AC1F3C221515CC84070470C000020FC
:1007800000100240120E000812A185B00FC98DE8BA
:100790000F0014A0144A006804905168134801F037
:1007A0000C03042B10D0082B0ED1C1F38343C903D3
:1007B0001DF803000AD5516804AAC1F34041515CF9
:1007C0000A4A5043B0FBF1F005B07047084948436E
:1007D000FAE7000002030405060708090A0B0C0DDE
:1007E0000E0F1010010200000010024000127A00EB
:1007F00000093D002DE9F84F040070D02078C04D6D
:10080000C00749D06868C0F38100012807D0686834
:10081000C0F38100022809D16868C00306D52868A2
:10082000800339D560680028E7D035E06068B0F50E
:10083000803F0BD010B1B0F5A02F11D0286820F464
:1008400080302860286820F4802002E0286840F486
:1008500080302860606890B1FFF750FE06460AE0DD
:10086000286840F480202860F0E700BFFFF746FECC
:10087000801B642873D828688003F7D50CE0FFF745
:100880003DFE064605E000BFFFF738FE801B6428EA
:10089000F0D828688003F7D420789A4E80074FF06C
:1008A00001094FF0000839D5686810F00C0F07D027
:1008B0006868C0F38100022809D16868C00306D4C3
:1008C0002868800714D52069012808D110E0206924
:1008D000B0B1C6F80090FFF711FE074605E00AE147
:1008E000FFF70CFEC01B0228C4D828688007F7D584
:1008F0002868616920F0F80040EAC10028600DE036
:10090000C6F80080FFF7FAFD074604E0FFF7F6FDA2
:10091000C01B022823D828688007F7D42078000756
:100920002CD57948A169D9B1C0F80090FFF7E6FD50
:10093000074604E0FFF7E2FDC01B02280FD8686AF3
:100940008007F7D571484FF4FA510068B0FBF1F019
:10095000009000BF0098411E0091FAD20EE080E0A6
:10096000C0F80080FFF7CAFD074604E0FFF7C6FDA8
:10097000C01B022875D8686A8007F7D42078400722
:1009800060D5E8690027C00008D4E86940F08050CD
:10099000E861E869012700F0805000905C48016838
:1009A000C90513D40168834641F480710160FFF7E3
:1009B000A5FD824606E000BFFFF7A0FDA0EB0A0000
:1009C00064284ED8DBF80000C005F5D5E0680128A2
:1009D0000AD008B1052813D0286A20F00100286247
:1009E000286A20F0040002E0286A40F00100286232
:1009F000E06841F2883B98B1FFF780FD82460BE04A
:100A0000286A40F004002862EEE700BFFFF776FD99
:100A1000A0EB0A0159455AD8286A8007F6D50CE0A0
:100A2000FFF76CFD824605E0FFF768FDA0EB0A01C9
:100A300059454CD8286A8007F6D41FB1E86920F0E0
:100A40008050E861E06988B36968C1F381010229D7
:100A500044D00228C6F8608004D0FFF74FFD04465A
:100A600038E034E0FFF74AFD074604E0FFF746FDB3
:100A7000C01B02282BD828688001F7D4206AB0F563
:100A8000803F05D16868A16820F4003008436860A1
:100A9000D4E908010843696821F4741108436860C7
:100AA000C6F86090FFF72AFD044606E025E000BF87
:100AB000FFF724FD001B022809D828688001F7D51C
:100AC0001BE000BFFFF71AFD001B022802D903201C
:100AD000BDE8F88F28688001F4D40EE00128F7D033
:100AE0006868226A00F48031914204D1616A00F49E
:100AF0007010884201D00120EAE70020E8E70000FA
:100B00000010024000004242800442420C000020DB
:100B10000070004010B5401EB0F1807F01D301206D
:100B200010BD4FF0E02460610F21601700F044F920
:100B30000020A06107202061002010BD70B50400D6
:100B400004D094F83D00002510B106E0012070BDEE
:100B500084F83C50204600F023F8242084F83D001F
:100B60002068C16821F40051C160204600F0B4F84B
:100B70002068016921F4904101612068416921F0F8
:100B80002A0141612068C16841F40051C1602564B7
:100B9000202084F83D0084F83E00002070BD000055
:100BA00030B585B000240094019402940394006849
:100BB0001449884224D11448816941F480418161FB
:100BC000816901F480410491816941F004018161EE
:100BD00080690E4D00F0040004904FF40070009006
:100BE000022001900320039069462846FFF78AFB04
:100BF0002815CDE90004694628460294FFF782FBD8
:100C000005B030BD0038014000100240000801402E
:100C1000FEE70000054808B5816941F004018161E3
:100C2000806900F00400009008BD00000010024040
:100C30000C4810B50A4901604FF4E13141600021D0
:100C400081600C22C160C0E904128161C161FFF7BB
:100C500075FF002803D0BDE81040FFF750BB10BD62
:100C600000380140100000207047FEE7FEE7FEE775
:100C700070477047FFF748BC30B58FB028216846F1
:100C8000FFF7C6FA14210AA8FFF7C2FA01210804E7
:100C9000CDE900100024029402250491CDE907500B
:100CA0004FF4E01009906846FFF7A4FD08B172B652
:100CB000FEE70F20CDE90A054FF48060CDE90C4036
:100CC00002210AA80E94FFF7A9FC002801D072B6F1
:100CD000FEE70FB030BD704770B50446006801698B
:100CE000E26821F44051114301612169A068084381
:100CF000616908432168CA6841F20C639A43024360
:100D0000CA6020684169A26921F4407111434161C0
:100D10001E492068884202D1FFF726FD01E0FFF757
:100D200013FD00EBC00101EB00126068642180003C
:100D3000B2FBF0F3B3FBF1F36FF018067343B2FBB1
:100D4000F0F5B2FBF0F605EB8305322303EB051556
:100D5000B5FBF1F5B6FBF1F605F0F00505EB061570
:100D6000B2FBF0F6B2FBF0F0B0FBF1F06FF018025E
:100D7000504306EB800003EB0010B0FBF1F021685C
:100D800000F00F002844886070BD0000003801406A
:100D9000FEE70000024901608021416070470000C9
:100DA000240E000800B50A46FFF7F4FF01498260EF
:100DB000016000BD300E00080907090E002804DBA1
:100DC00000F1E02080F80014704700F00F0000F1FF
:100DD000E02080F8141D704701490248FFF7E2BF88
:100DE0001000002054000020FFF796FBFFF744FF9F
:100DF000FFF710FFFFF71CFFFFF736FFFFF735FF88
:100E0000FCE70000000000000000010203040607E8
:100E100008090000000001020304000000000000B7
:100E200000000000000000000000000000000000C2
:100E300000000000580E0008000000201000000014
:100E40006C010008680E000810000020B0260000A9
:100E50008801000885FFFFFF01000000100000006E
:080E6000000000000024F40072
:0400000508000131BD
:00000001FF
